:030000000219FDE5
:03000B000200AA46
:03002B0002015C73
:03005B000202F6A8
:030073000202E3A3
:1000800002030406080C10182030406080040608A3
:100090000C10182030406080A0C00003070F1F0D17
:1000A0000D04050D050305030302C2AFC0D0C0E077
:1000B000206214E5256009E473E525F4F58AD2622F
:1000C000D0E0D0D0D2AF3285268AC262E526F46075
:1000D0002F30682520720DD0E0D0D0C293C295C2D7
:1000E00097D2AF32C293C295C297206F0C20650998
:1000F000740AD5E0FDE57B4290D0E0D0D0D2AF329B
:10010000758A00C28DD26201F901B9306805206597
:1001100002D29301B9306805206502D29501B93049
:100120006805206502D29701B9C29230680A20653D
:10013000077408D5E0FDD29301B9C29430680A2053
:1001400065077408D5E0FDD29501B9C29630680AFA
:100150002065077408D5E0FDD29701B9C2AFC2ADE2
:1001600053E6EFC0D0C0E0D2D3D2AFC2CEE52A6012
:100170000720744F152A21C37800790020742EE5DA
:1001800080307E01F430E30278FF53DACF207E0323
:1001900043DA20307E0343DA10C2D8C271E58030E2
:1001A0007E01F430E30279FFC3E89970CB3061033C
:1001B000752A18207403752A18885CD270E86003C9
:1001C000755F0020740DE52B6004152B21D343DAF5
:1001D00001C2D82070024142A85C206102C2702096
:1001E00074367982B70431C3E894F0400374F0F8B0
:1001F000E8C4540F28F87984B703024118C313C325
:10020000138721200802C313200A06C3C898F841A7
:100210001828F8500374FFF88822E52D5406602250
:10022000206B1FE536C333C333F8E564C313C31330
:10023000F9C3952240028922E82522F52250037550
:1002400022FF7882B60459852224A824C3E5249588
:10025000614002A861C3E895634002A8638825E570
:100260006670024193C3E8AA669A5003E8FAE4F97B
:10027000EAC333FBE568F45B29400D2567F8E567C1
:1002800060021567400B41930AC3E5679A50020567
:100290006778FF8826C26FC3E52694F84002D26FC4
:1002A00020CF0AD0E0D0D043E610D2AD32C2CF0585
:1002B0003A7801E52A6005307402152AC3E55C949A
:1002C000014005755F0041D9756000756900E55F03
:1002D0002401F55F5003755FFFD0E0D0D043E610F6
:1002E000D2AD32C2AF53E67F7592FA7593FFC2600A
:1002F000759104D2AF32C2AF53E6EFC2ADC0D0C0E9
:10030000E0C0F0D2D3D2AFA8FBA9FCC2D8307102B2
:10031000615D53DACF207E0343DA10307E0343DA87
:1003200020D271E580307E01F420E3026134882719
:100330008928A18A53DACF207E0343DA20307E0356
:1003400043DA10C2D8C271307402A1767800E58019
:10035000307E01F430E302A176885CA15E53DACFEF
:10036000207E0343DA20307E0343DA10C27120611D
:1003700002813653DACF207E0343DA10307E034306
:10038000DA20C2D8D27188578958C3E89555F8E960
:100390009556F97B007E087A00C3E8948CE99400B6
:1003A0005005755B008128882178A2E6A821605558
:1003B000C3E894C8E994005008E4D2E4FB7A0A81C7
:1003C00003C3E89468E994015008E4D2E3FB7A0F90
:1003D0008103C3E894D0E994025008E4D2E2FB7AA6
:1003E0001E8103C3E894A0E994055008E4D2E1FB20
:1003F0007A3C8103C3E89498E994085008E4D2E079
:10040000FB7A787E00C3E89559FCE9955AFD30E700
:100410000AECF42401FCEDF43400FD755B00C3EC40
:100420009AED9E5003755B018859895A8557558509
:1004300058567802A15EC3E89527F8E99528F93067
:100440007C02A142307B02A142307A02A13B20759E
:10045000028159E9FDE8FC8178E9C313F9E813F852
:10046000307902A13BE9C313F9E813F8307802A10F
:0F0470003BE9C313FDE813FC20612CC3EC941C83
:10047F00ED94024002818FED701EC3EC94C85018AA
:10048F000529E52970021529C3E529940A5002A10F
:10049F0076755C00D270A176E529600215297888FF
:1004AF00E6F97400207F087896B90302789EE62457
:1004BF00FAFEE43400FFC3EC9EFCED9FFD9208B9F9
:1004CF000310A2085007207609D27681E130760218
:1004DF00C276A2085016B9030DECF42401FCEDF41A
:1004EF003400FD0204FB78007900A142B90315EC3A
:1004FF0033FCED33FDC3EC940AFCED9400FD500486
:10050F007C007D00C3EC94FFED9400400678FF79EA
:10051F0000A142EC8572F0A4C5F0A2F733F8790080
:10052F00400302055E78FF790002055EE9C313F907
:10053F00E813F8307C0EE9600278FFC3E81338F84F
:10054F00E43400F9C3E894FFE99400400278FF888F
:10055F005CD270206102A176741FF4552F4BF52FDA
:10056F00C274EB7002D274752A18307403752A0A9C
:10057F00306102A18A20740353DAFE207403752BB5
:10058F0006D0F0D0E0D0D0D2AD43E61032790102E0
:10059F0005BA79030205BA790A0205BA791E02056E
:1005AF00BA79640205BA79C80205BA7817E4D5E0BA
:1005BF00FDD8FAD9F6227A147B780205E17A107BFE
:1005CF008C0205E17A0D7BB40205E17A0B7BC80240
:1005DF0005E1E573D5E001227902E4C294D5E0FD8F
:1005EF00D295D5E0FDC295D5E0FDD294D5E0FDE9D9
:1005FF0020E002D29330E002D297E573D5E0FDE917
:10060F0020E002C29330E002C2977496D5E0FDD984
:10061F00C9EAF8D5E0FDD8FBDBB8C29422C37C0051
:10062F007D0075F00005F0EA33FAEB33FB50F6EB83
:10063F0013FBEA13FAC3E9FFE8FEE89AF8E99BF91E
:10064F005004EFF9EEF8B3EC33FCED33FDD5F0DFEA
:10065F00EDF9ECF822E889F08A20D2D4F8A9F07BE2
:10066F000030F70B7BFFF42401F8E9F43400F9E8CC
:10067F008520F0A4ADF0F8E98520F0A4AFF0FEEDF1
:10068F002EF974003FFA7C04C3EA13FAE913F9E870
:10069F0013F8DCF48BF030F70AE8F42401F8E9F4EE
:1006AF003400F9E889F0C2D4F8A9F0227882B604B0
:1006BF0003020716C3E55C940140030206E085229E
:1006CF0024E4F544F545F546F547F548C26E0207B3
:1006DF00167882E6FCD26EE522F523783879C7AA20
:1006EF0040AB41C3EB13FBEA13FAEC146013C3EBFB
:1006FF0013FBEA13FAEC14146007C3EB13FBEA13B2
:10070F00FAD12C8844894522C3E5449523F8E54561
:10071F009400F9500CC3E89480E994FF4016020747
:10072F0047C3E8947FE994005003020747787F7925
:10073F0000020747788079FF8849894A22E54925D1
:10074F0046F8E54A3547F9854A20E4300701F43584
:10075F0048FA30E709C3EA94F04015020785C3EA67
:10076F00940F500302078578FF79FF7A0F020785F0
:10077F00780079007AF0C3E5249561500AC37401BB
:10078F009524500B0207A3E54A20E70E0207A3E5C5
:10079F004A30E706884689478A482278A5E6FAC391
:1007AF00E54933F8E54A33F9D164E930E70BC3E89B
:1007BF009480E994FF4013E1DDC3E8947FE994004E
:1007CF005002E1DD787F7900E1DD788079FFE82064
:1007DF00E715C3E52398F84009C3E89401400302E5
:1007EF0008047801020804E8F424012523F84003E3
:1007FF0002080478FF884B2278A6E6FAA847A94892
:10080F00120664E930E70CC3E89401E994FF40163F
:10081F00020839C3E894FFE99400500302083978BD
:10082F00FF7900020839780179FFE920E715C3E560
:10083F004B98F84009C3E89401400302086078011F
:10084F00020860E8F42401254BF8400302086078A1
:10085F00FF88242278FF20692879A1E76023E541EA
:0E086F00601F74FF8541F0848539F0306A0304
:10087D0075F005A4F8C5F0600278FFC3E8956450E3
:10088D0002A864886322C3E5409440E5419401E5E4
:10089D006350031401A4046002F563220208AC2224
:1008AD0075E890227883E6FF30EDF9A8BDA9BE0565
:1008BD0070C3E57094084052757000E9FA79A0E7AD
:1008CD006044EA7007E571601B0208E5C3E89571A5
:1008DD006010E5715006600C140208F10460F90215
:1008ED0008F1E571F571C394A8401B7561C0C394FF
:1008FD00054013756180C39405400B756140C39429
:10090D0005400375610075BB0122E561241050029D
:10091D0074FFF5617982B70402213EC3A861E52415
:10092D00985002A824C3E895634002A863882588DF
:10093D0026E570B4070375BB1E22743279A787F0C4
:10094D00A4C5F0A2F733F8C3E895614002A8618809
:10095D00228824882588268864227540007541F0F8
:10096D0022C2AF75C820A8CCA9CDAA3A30CF010AB2
:10097D0075C824D2AFAB3BAC3C883B893CC3E89BEC
:10098D00F8E99C206908F9306602417F21D9AD3D17
:10099D008A3DF9EA9DFA600678FF79FF21BEAE3EE9
:1009AD00AF3F8B3E8C3FA83BA93CC3E89EF8E99F27
:1009BD00F9C3E54113FBE54013FAE82AF540E93B9D
:1009CD00F54150067540FF7541FF4126AA40AB41E8
:1009DD00AC40AD417E047F02C3EB9404400D1E1F5D
:1009ED00C3EB94084005206A021E1FC3ED13FDECF6
:1009FD0013FCDEF7C3EA9CFAEB9DFBEF6009C3E93C
:100A0D0013F9E813F8DFF7EA28FAEB39FB8A408B84
:100A1D004150067BFF8B408B41C3EB94025002D2B9
:100A2D00663069047F0341517892E6FFC3E5379440
:100A3D008240110FC3E53794A040010FC3EF940618
:100A4D0040027F057E02E541C4540FF9E541C454CF
:100A5D00F0F8E540C4540F28F8C3E89EFAE9940075
:100A6D00FB4009C3EA9402EB940050047A02E4FBC4
:100A7D0041CBAA40AB41EBC4FEEAC4540F4EFCC3BC
:100A8D00EA9CFAEB9400FBC3E813C313F8EA28FAC7
:100A9D00EB3400FB8A408B41C3EB94024002C266EB
:100AAD007802EBC4FE7B00EAC4540F4EFAC3EA98F9
:100ABD00FA4005C3940250027A027892E6FF306044
:100ACD000241CB855192855293D26043E680C3E4B7
:100ADD009AF8E49BF93066026157E8FAE9FBD3E92D
:100AED0013FDE813FC88518952C3EF94036038EF6E
:100AFD0020E00DE82CF8E93DF9ECFAEDFB020B20B6
:100B0D00E828F8E939F9C3E82402F8E93400F97A5C
:100B1D00FE7BFFC3EF9403400E8A538B54884D899F
:100B2D004E8C4F8D50618B885389548A4D8B4E8CD2
:100B3D004F8D503069127553F07554FF754FF07528
:100B4D0050FF7551F07552FF618BE8FAD3E813FC35
:100B5D008851C3EF94036020EF20E007E82CF8ECF8
:100B6D00FA6177E8282402F87AFEC3EF940340086F
:100B7D008A53884D8C4F618B88538A4D8C4FE56815
:100B8D00C3335002646BF5683060026195753402B1
:100B9D00D26043E680E52D54066034A840A941C3D8
:100BAD00E913F9E813F8C3E913F9E813F830690408
:100BBD00E92440F9C2AF53E67F759100C3E498F57F
:100BCD0094E499F595759104D26043E680D2AF22F5
:100BDD00D264754300752000306C03752040020B04
:100BED00FCD264754300752040306C03752000788D
:100BFD00017901206620E52D54066002C264791446
:100C0D00E541C313700104F8C39414400278143005
:100C1D006904781B791B206010E543600C30690373
:100C2D00D53404D26D81AF719D0543E59E7005E508
:100C3D009B020C43E59A5440B52002819930690915
:100C4D0008C3E899400118812320640A08C3E89974
:100C5D00400261FC8123C264C2AF53E67F759100EF
:0E0C6D003066127594007595F8759104D2608A
:100C7B0043E680D2AF61FCE5417EFFC3334005C341
:100C8B00334001FEC3E49E759400F5958176C3E570
:100C9B00339401500261FC30640261FCD80281ADD7
:100CAB008123C26DC2AF53E67F7591008553948546
:100CBB005495759104854D92854E93D26043E68091
:100CCB00D2AFE52D54066008206A020533020CEB07
:100CDB00306D0D206C0A206407158115810215CD2E
:100CEB002278003064027801E53775F007A4F9E546
:100CFB00F028F5F0E9A2F013A2F113A2F213F537E5
:100D0B00C394785003753778C3E53795384008D2CC
:100D1B0065C293C295C297306002A122854F92851E
:100D2B005093D26043E68022207D19C2AF754202F8
:100D3B00C294D292306202D297D2AF759F33759E16
:100D4B0000020F35C2AF754202C294D296306202D6
:100D5B00D293D2AF759F33759E00020F353072431D
:100D6B00207D20C2AF75420390013A757B10C2976C
:100D7B00C296306204D295A186D294D2AF759E23CF
:100D8B00020F35C2AF75420390013A757B10C293C7
:100D9B00C292306204D295A1A6D294D2AF759E2294
:100DAB00020F35207D17C2AF754203900115C29714
:100DBB00306202D295D2AF759E23020F35C2AF754A
:100DCB004203900115C293306202D295D2AF759E49
:100DDB0022020F35207D16C2AF754204C292D29605
:100DEB00306202D295D2AF759E22020F35C2AF751B
:100DFB004204C296D292306202D295D2AF759E2334
:100E0B00020F35307249207D23C2AF754205900128
:100E1B0029757B04C295C294306204D293C12CD243
:100E2B0092D2AF759F33759E00020F35C2AF7542DC
:100E3B000590014B757B40C295C294306204D297EA
:100E4B00C14FD296D2AF759F33759E00020F3520DE
:100E5B007D1AC2AF75420590010BC295306202D26A
:100E6B0093D2AF759F33759E00020F35C2AF75429B
:100E7B000590011FC2953062E8D297D2AF759F33B0
:100E8B00759E00020F35207D16C2AF754206C296C5
:100E9B00D294306202D293D2AF759E23020F35C229
:100EAB00AF754206C292D294306202D297D2AF751E
:100EBB009E22020F35307244207D20C2AF75420155
:100ECB0090014B757B40C293C292306204D297C1A2
:100EDB00DED296D2AF759E22020F35C2AF7542019C
:100EEB00900129757B04C297C296306205D293029A
:100EFB000EFFD292D2AF759E23020F35207D17C203
:100F0B00AF75420190011FC293306202D297D2AFEC
:100F1B00759E22020F35C2AF75420190010BC2972D
:100F2B00306202D293D2AF759E23C2652290010923
:100F3B00757B00C293C295C297C292C294C296C2ED
:100F4B006222788076090876090876040876FF080D
:100F5B0076030876FF08760708760308760108768D
:100F6B0001788C76010876FF0876FF0876FF087605
:100F7B00FF0876FF0876030876FF0876FF0876FFF2
:100F8B000876250876D00876280876500876040867
:100F9B0076FF08760208760008767A0876FF0876E0
:100FAB000108760108760008760308760022788718
:100FBB00E6FFC272BF0302D2727888E6C394036065
:100FCB0008C27DE630E102D27DC27E7889E630E14F
:100FDB0002D27EC3EF94026008758E01D273020FAA
:100FEB00F1758E00C273227880E61490008093789E
:100FFB00A5F67881E6149000809378A6F67886E6BD
:10100B001490008D9378A7F67886E6F539C3940291
:10101B005003753902789CE67538FFB402037538B6
:10102B00A0B4030375388278A3E61490009A93F565
:10103B0066120F3822227896E6FA7897E6FB7888C4
:10104B00E6B40305C3EB940EFB307F047A007BFF01
:10105B00C3EB9AFCC3948250027C827572000572BA
:0F106B00EC8572F0A4C3E5F0947D40F222D27FB1
:10107A0011411205AB1205AB7A007B007C101205F8
:10108A00A1E55C2AFA74003BFBDCF37C04C3EB1396
:10109A00FBEA13FADCF7FEC27F114122757C007568
:1010AA007D00E5EF20E6037520000520903DFFE571
:1010BA0020146006901FFF1460009304600375EF0C
:1010CA001653D9BF7581C043FF8012059C75EF0680
:1010DA0043B203E5B3240220E70DF521E5B120E090
:1010EA00068521B343B101120F3875800875A40033
:1010FA0075F1FF75D4F775900275A5FC75F2FC754C
:10110A00D50075A0FD75A60275F30275D60075B0F7
:10111A00FF75A70175F4FF75E241120F38E4F8F67E
:10112A00D8FD756801120F4D12161E7898867375D0
:10113A003001C2AF1205B51205C51205AB1205CCB6
:10114A001205AB1205D31205ABC2AF757C00757DD3
:10115A000078FA79FA308307D9FBD8F7021C001213
:10116A000FB9120FF21140114178988673120F3895
:10117A0075881075890275C82475910475D84075EB
:10118A00A82275B80275E690759B80759D00759AC0
:10119A0080759C0075D10E75BC5875BB0175BA1F58
:1011AA0075E88012059CD2AF1208A975360053DA89
:1011BA00CF207E0343DA20307E0343DA1043DA017C
:1011CA00C2D8C2711205B5D2617B037A0CE55B7095
:1011DA00077A0CDB030211531205AB2070030211CC
:1011EA0053C270E55CC3940240E1E52F541F855E4B
:1011FA005DF55EB55DD5DAD5C26153DACF207E03DF
:10120A0043DA20307E0343DA10C2D8C27178A2E6EC
:10121A007008D274E52F54E0F52FC27575290012B3
:10122A0005B0307409C3E529940A4002D275120543
:10123A00A178023074027800C3E55C9840F0C2AF2E
:10124A001205C51205C51205C5D2AF1205B5754CF2
:10125A00007888E6B40302614E1205A1788CE6C3D1
:10126A009401500302134EE530C394015003021354
:10127A004E757CA5757DF1207435C3E55C94FF50ED
:10128A000302134EC2AF1205DAD2AF1205B0C3E59C
:10129A005C940150EFC2AF1205C51205A61205C52E
:1012AA00D2AF1205B0C3E55C94FF40E90217D67FBE
:1012BA0002D27F11411205B0C2AFC27F1141AE5CAA
:1012CA00C3E55C947FD2AF5002615E12059CC2AF47
:1012DA001205DAD2AFDFDA1178C3EE7897F6120583
:1012EA00B51217597F0AD27F11411205B0C2AFC297
:1012FA007F1141AE5CC3E55C947FD2AF50E6120524
:10130A009CC2AF1205C51205A61205C5D2AFDFD61B
:10131A001178EE24037896F6F87997E7C394824019
:10132A0003985006E824827897F61205B512166CCF
:10133A001217881205B01141C3E55C94FF500241AF
:10134A007B0217D6757C00757D00C3E55C954C4021
:10135A0003855C4C1205B078017988E7B4030278FA
:10136A0005C3E55C984002415BC2AF1205DA12057B
:10137A00DA1205DAD2AF1205B5753000E4F531F5A7
:10138A00320531E531F4703F0532789AE67819145E
:10139A006012783214600D787D14600878FA14604F
:1013AA0003753200C3E53298401D120F3812059CAE
:1013BA00153275310078998673C2AF1205DAD2AF49
:1013CA00789886731205B01205A6E52A700530745E
:1013DA0002215378012074027806C3E55C9840A183
:1013EA007888E6C3940360031205B0E52A70030205
:1013FA001153C2AF120F38E4F522F523F524F5256F
:10140A00F526F567D2AF7885E6C333F565E4F5448A
:10141A00F545F546F547F548F570F52CF52DF53700
:10142A0075700875BB1E12059C1208AD30EDFDA83B
:10143A00BDA9BEE97001F888711208B17570087506
:10144A00BB1E120FB9C2AF7561FF1209478522612F
:10145A00852262852263D2AF752201752401752522
:0D146A0001752601856069756A017888E6C4
:10147700B40307C27D307602D27DD268D269753354
:1014870000120E91120EC012096712096E12096737
:1014970012096E120967120BEE1206BB120CEC1240
:1014A7000D3312096E120BDD306E0312071720661B
:1014B70003120863306603120893120CEC120D68CE
:1014C70012096E120BEE306E0312074C120CEC125F
:1014D7000DDF12096E120BDD306E031207AA120C14
:1014E700EC120E0E12096E120BEE306E0312080785
:1014F700120CEC120E9112096E1208AD120BDD12CE
:101507000CEC120EC01208B112096E3069328564F4
:1015170061856462856069756A0179187A0CC3E52B
:101527003399400FC269D26A8A35856461856463DD
:10153700021547C3E55C9401400302149D0215D5CB
:10154700306A25206C22E535147006C26AD26B8199
:101557009DF535C3E55C9401400302149D7888E648
:10156700C3940360030215D575360078FA79A4E7AA
:1015770060027803C3E55F985054307404E52A602D
:101587004D7888E6B40317207D05207607A1A5309E
:101597007602A1A5206C07D26C85646181DC78F0A6
:1015A700306C058564617820C3E541985002819DC0
:1015B700306C1BC26CC27D307602D27DD26A753523
:1015C70012856461819D0536E55C6002A1D8753698
:1015D70000C2AF120F387887E6FE7602120FB9788D
:1015E70087EEF6E4F522F523F524F525F526F565CE
:1015F700752C00752D00D2AF1205B0120F3878A4E4
:10160700E66006D293D295D297307409C3E5369433
:1016170004400221536186901A0D78201216AEE518
:1016270020B4550CA31216AEE520B4AA0302164C3B
:10163700757CA5757DF1120F4D12166C757C0075C2
:101647007D0002166B901A0378807B0A1216AEA3F0
:1016570008DBF9901A0F788C7B191216AEA308DBFA
:10166700F9901A2822C2AF1216F11216CE901A005C
:10167700740E1216B3A374091216B3A374151216B7
:10168700B3901A0378807B0A1216B2A308DBF9908D
:101697001A0F788C7B191216B2A308DBF9121704FC
:1016A7001216E2901A2822E493F622E6438F01539A
:1016B7008FFDFFC3E583941C400122EF857CB7852E
:1016C7007DB7F0538FFE22438F02438F01857CB78E
:1016D700857DB7901A0DF0538FFC22901A0D745523
:1016E700D1B3901A0E74AAD1B3227A3079D0782068
:1016F700901A40D1AEE520F709A3DAF7227A3079BC
:10170700D0901A40E7D1B309A3DAF922AB74A875D0
:10171700BB01027980BB02027981BB03027982BBDC
:1017270004027984BB05027986BB06027992BB075E
:10173700027987BB080279A3BB0902799CBB0A021D
:101747007988BB0B027989E8F7227C051205B5DC9D
:10175700FB22C2AF1205C51205CC1205D31205DA5A
:101767001205A61205C51205CC1205D31205DA1209
:1017770005A61205C51205CC1205D31205DAD2AF9C
:1017870022C2AF1205DA1205D31205CC1205C51213
:1017970005A61205DA1205D31205CC1205C51205E6
:1017A700A61205DA1205D31205CC1205C5D2AF224F
:1017B700AE74AF75C2AF1205C51205C51205C512C5
:1017C70005A6DEF21205DA1205A6DFF8D2AF22F17E
:1017D70059F151F151757401757501757600F1B7BD
:1017E7007C05AD5C1205B5C3ED955C70F5C3E55C92
:1017F7009401400AC3E55C94FF403702181612179C
:101807001312166C121759C2AF75EF16121751DC67
:10181700D10576C3E5769403500280C212175105AD
:1018270075E5741490009F93F808C3E57598500206
:1018370080A91217511217510574C3E574940C50FF
:10184700028095120F4D12166CC2AF75EF16121764
:01185700513F
:0319FD000210A62F
:101A00000E0915090904FF03FF0703010155AA0187
:101A1000FFFFFFFFFF03FFFFFF25D0285004FF0259
:091A2000007AFF0101000300FF40
:101A400023506C6174696E756D31353041232020EF
:101A500023424C48454C4923463331302320202033
:101A60002020202020202020202020202020202076
:101C0000C2AFC2D353D9BF7581C043B20343FF8073
:101C1000752438752503B1DC7529A5752AF175E29F
:101C20004043F10853A4F775D4FFD2837DFA7803BB
:101C300079E67C10752200752300901DE97B0675FE
:101C400024987525013083028145208308D8FBD96B
:101C5000F9DCF781B7308308D8FBD9F9DCF781B715
:101C6000B19CE493A3C39A6004DDC381B7DBDBB10D
:101C70008E6002812E7B08E493FAA3B16FDBF87AC1
:101C800030B16F752200752300B18EEAFCEBFDC305
:101C9000ED94FE400EB18E8A278B28ED30E0048A49
:101CA000828B83B18E7AC270D8C3ED94FE601950D6
:101CB000CEBD002BEC600F7520007521FF7529004B
:101CC000752A000200008100A827A9280809D80465
:101CD000D90281DCB192EA89AAF281CE0D81A3C337
:101CE000ED94035053EDA2E092007AC5C3E58294CF
:101CF00000E583941C508A200010438F02438F011B
:101D00008529B7852AB7F0300029A827A92808090E
:101D1000438F01538FFDD804D902A133C3E58394C7
:101D20001C4003A3A11689AAE28529B7852AB7F02A
:101D3000A3A116538FFC817F7AC1BD030CE493A34A
:101D4000FAB153DCF8B14B817F8181AA22AB23B178
:101D50006FEBFAEA6222752608C3E52313F523E543
:101D60002213F52250066323A0632201D526EAB18F
:101D7000DCB1DC75260AEAF4200102D283300102CC
:101D8000C283B1DCC3134002C201D526EB22B1925B
:101D9000EAFB208302A192308302A197752608AE48
:101DA00024AF25C3EF13FFEE13FEB1E0B1DCC3EAAD
:101DB000133083024480FA30E703632201C3E52332
:101DC00013F523E52213F52250066323A0632201B5
:101DD000D526D9E52265236523F52222AE24AF2539
:101DE0000E0FDEFEDFFCD20122424C48656C6934E6
:071DF000373164F310060116
:00000001FF
